:1000000090C001C063C01FB6816022BE02E008BF7D
:1000100002E009BF01E003BF00E00BBF1FBE18955F
:100020004094042D0329057008BB4A9519F540E258
:10003000503019F487FD53951DC0513019F4332405
:10004000539518C05A3031F4002760FF0FEF302E5F
:10005000539510C05B3039F40FEF302E539560E0AC
:1000600050E08F7707C00027779510F40FEF639566
:10007000302E539508951A9541F5203039F4B199F1
:1000800002C011E022C0239514E01FC0213029F4E2
:10009000B19B19C0239518E018C02A3069F4B199B2
:1000A00012C0903280F439939395C03808F0C0E6BE
:1000B00020E011E08E7F09C00894B19988943795AB
:1000C000239518E002C020E011E008951FB622BE7B
:1000D000A7DFD1DF1FBE1895A0E0A1BDA3E2A5BF99
:1000E000A4ED2A2E11E020E0AFEF3A2EA0E04A2E38
:1000F00040E250E060E080E090E0C0E6D0E0E0E682
:10010000F0E0A5E0A7BBA5E0A8BBA0E0A3BFA0E0EE
:10011000A9BFA2E0A8BF22BEA0E4AABFA0E4ABBFD3
:100120000895A0E0A4BFAFEDADBFD6DF789487FD02
:10013000FECF903041F0A1919A95E03808F0E0E6CA
:100140007A2F8068F4CF80FDF2CFA0E0A3BFA0E0BB
:10015000A9BFA2E0A8BF22BEA0E4AABFA0E4ABBF93
:040160008895E5CFCA
:00000001FF
